BL51 BANKED LINKER/LOCATER V6.22                                                        04/27/2022  11:38:43  PAGE 1


BL51 BANKED LINKER/LOCATER V6.22, INVOKED BY:
C:\KEIL_V5\C51\BIN\BL51.EXE .\Objects\main.obj, .\Objects\OPTIONS_SN8F5835.obj TO .\Objects\SN8F5835_Test Code PRINT (.\
>> Listings\SN8F5835_Test Code.m51) RAMSIZE (256)


MEMORY MODEL: SMALL


INPUT MODULES INCLUDED:
  .\Objects\main.obj (MAIN)
  .\Objects\OPTIONS_SN8F5835.obj (OPTIONS_SN8F5835)
  C:\KEIL_V5\C51\LIB\C51S.LIB (?C_STARTUP)


LINK MAP OF MODULE:  .\Objects\SN8F5835_Test Code (MAIN)


            TYPE    BASE      LENGTH    RELOCATION   SEGMENT NAME
            -----------------------------------------------------

            * * * * * * *   D A T A   M E M O R Y   * * * * * * *
            REG     0000H     0008H     ABSOLUTE     "REG BANK 0"
            DATA    0008H     0008H     UNIT         _DATA_GROUP_
            IDATA   0010H     0001H     UNIT         ?STACK

            * * * * * * *  X D A T A   M E M O R Y  * * * * * * *
                    0000H     F000H                  *** GAP ***
            XDATA   F000H     0001H     ABSOLUTE     
            XDATA   F001H     0001H     ABSOLUTE     
            XDATA   F002H     0001H     ABSOLUTE     
            XDATA   F003H     0001H     ABSOLUTE     
            XDATA   F004H     0001H     ABSOLUTE     
            XDATA   F005H     0001H     ABSOLUTE     
            XDATA   F006H     0001H     ABSOLUTE     
            XDATA   F007H     0001H     ABSOLUTE     
            XDATA   F008H     0001H     ABSOLUTE     
            XDATA   F009H     0001H     ABSOLUTE     
            XDATA   F00AH     0001H     ABSOLUTE     
            XDATA   F00BH     0001H     ABSOLUTE     
            XDATA   F00CH     0001H     ABSOLUTE     
            XDATA   F00DH     0001H     ABSOLUTE     
            XDATA   F00EH     0001H     ABSOLUTE     
            XDATA   F00FH     0001H     ABSOLUTE     
            XDATA   F010H     0001H     ABSOLUTE     
            XDATA   F011H     0001H     ABSOLUTE     
            XDATA   F012H     0001H     ABSOLUTE     
            XDATA   F013H     0001H     ABSOLUTE     
            XDATA   F014H     0001H     ABSOLUTE     
                    F015H     0001H                  *** GAP ***
            XDATA   F016H     0001H     ABSOLUTE     
            XDATA   F017H     0001H     ABSOLUTE     
            XDATA   F018H     0001H     ABSOLUTE     
            XDATA   F019H     0001H     ABSOLUTE     
            XDATA   F01AH     0001H     ABSOLUTE     
            XDATA   F01BH     0001H     ABSOLUTE     
            XDATA   F01CH     0001H     ABSOLUTE     
            XDATA   F01DH     0001H     ABSOLUTE     
            XDATA   F01EH     0001H     ABSOLUTE     
BL51 BANKED LINKER/LOCATER V6.22                                                      04/27/2022  11:38:43  PAGE 2


            XDATA   F01FH     0001H     ABSOLUTE     
            XDATA   F020H     0001H     ABSOLUTE     
            XDATA   F021H     0001H     ABSOLUTE     
            XDATA   F022H     0001H     ABSOLUTE     
            XDATA   F023H     0001H     ABSOLUTE     
            XDATA   F024H     0001H     ABSOLUTE     
            XDATA   F025H     0001H     ABSOLUTE     
            XDATA   F026H     0001H     ABSOLUTE     
            XDATA   F027H     0001H     ABSOLUTE     
            XDATA   F028H     0001H     ABSOLUTE     
            XDATA   F029H     0001H     ABSOLUTE     
                    F02AH     0001H                  *** GAP ***
            XDATA   F02BH     0001H     ABSOLUTE     
            XDATA   F02CH     0001H     ABSOLUTE     
            XDATA   F02DH     0001H     ABSOLUTE     
            XDATA   F02EH     0001H     ABSOLUTE     
            XDATA   F02FH     0001H     ABSOLUTE     
            XDATA   F030H     0001H     ABSOLUTE     
            XDATA   F031H     0001H     ABSOLUTE     
            XDATA   F032H     0001H     ABSOLUTE     
            XDATA   F033H     0001H     ABSOLUTE     

            * * * * * * *   C O D E   M E M O R Y   * * * * * * *
            CODE    0000H     0003H     ABSOLUTE     
            CODE    0003H     0077H     UNIT         ?PR?MAIN?MAIN
            CODE    007AH     0019H     UNIT         ?PR?GPIO_INITIALIZATION?MAIN
            CODE    0093H     000CH     UNIT         ?C_C51STARTUP
                    009FH     7F51H                  *** GAP ***
            CODE    7FF0H     0002H     ABSOLUTE     
                    7FF2H     0004H                  *** GAP ***
            CODE    7FF6H     000AH     ABSOLUTE     



OVERLAY MAP OF MODULE:   .\Objects\SN8F5835_Test Code (MAIN)


SEGMENT                                DATA_GROUP 
  +--> CALLED SEGMENT                START    LENGTH
----------------------------------------------------
?C_C51STARTUP                        -----    -----
  +--> ?PR?MAIN?MAIN

?PR?MAIN?MAIN                        0008H    0008H
  +--> ?PR?GPIO_INITIALIZATION?MAIN



SYMBOL TABLE OF MODULE:  .\Objects\SN8F5835_Test Code (MAIN)

  VALUE           TYPE          NAME
  ----------------------------------

  -------         MODULE        MAIN
  C:0000H         SYMBOL        _ICE_DUMMY_
  X:F003H         PUBLIC        PW1YL
  X:F017H         PUBLIC        PW2YL
BL51 BANKED LINKER/LOCATER V6.22                                                      04/27/2022  11:38:43  PAGE 3


  D:00ADH         PUBLIC        CRCDATL
  D:0080H         PUBLIC        P0
  X:F031H         PUBLIC        PW3YL
  D:0090H         PUBLIC        P1
  D:00B0H         PUBLIC        P3
  D:00C8H         PUBLIC        P4
  D:00A0H         PUBLIC        TTCON
  D:00A8H         PUBLIC        IEN0
  D:00B8H         PUBLIC        IEN1
  X:F004H         PUBLIC        PW10DH
  X:F018H         PUBLIC        PW20DH
  X:F006H         PUBLIC        PW11DH
  X:F01AH         PUBLIC        PW21DH
  X:F00CH         PUBLIC        PW30DH
  X:F008H         PUBLIC        PW12DH
  X:F01CH         PUBLIC        PW22DH
  X:F00EH         PUBLIC        PW31DH
  X:F00AH         PUBLIC        PW13DH
  X:F01EH         PUBLIC        PW23DH
  X:F010H         PUBLIC        PW32DH
  X:F005H         PUBLIC        PW10DL
  X:F019H         PUBLIC        PW20DL
  X:F012H         PUBLIC        PW33DH
  X:F007H         PUBLIC        PW11DL
  X:F01BH         PUBLIC        PW21DL
  X:F00DH         PUBLIC        PW30DL
  X:F009H         PUBLIC        PW12DL
  X:F01DH         PUBLIC        PW22DL
  X:F00FH         PUBLIC        PW31DL
  X:F00BH         PUBLIC        PW13DL
  X:F01FH         PUBLIC        PW23DL
  X:F011H         PUBLIC        PW32DL
  X:F013H         PUBLIC        PW33DL
  X:F000H         PUBLIC        PW1M
  D:00ACH         PUBLIC        CRCM
  C:0003H         PUBLIC        main
  X:F014H         PUBLIC        PW2M
  X:F02DH         PUBLIC        HIDR
  X:F028H         PUBLIC        P0UR
  X:F001H         PUBLIC        PW3M
  X:F029H         PUBLIC        P1UR
  X:F02BH         PUBLIC        P3UR
  X:F02CH         PUBLIC        P4UR
  D:00D8H         PUBLIC        CSCON4
  B:0080H.0       PUBLIC        P00
  D:0088H         PUBLIC        TCON
  X:F027H         PUBLIC        TSWA
  X:F026H         PUBLIC        TSWB
  X:F025H         PUBLIC        TSWD
  D:00F9H         PUBLIC        P0M
  D:00FAH         PUBLIC        P1M
  D:00FBH         PUBLIC        P3M
  D:00FCH         PUBLIC        P4M
  X:F02EH         PUBLIC        CSADB1H
  X:F024H         PUBLIC        TSWY
  X:F032H         PUBLIC        CSADB2H
  X:F02FH         PUBLIC        CSADB1L
BL51 BANKED LINKER/LOCATER V6.22                                                      04/27/2022  11:38:43  PAGE 4


  X:F033H         PUBLIC        CSADB2L
  C:007AH         PUBLIC        GPIO_Initialization
  D:0098H         PUBLIC        S0CON
  X:F022H         PUBLIC        MINCS0H
  X:F020H         PUBLIC        MAXCS0H
  X:F023H         PUBLIC        MINCS0L
  X:F021H         PUBLIC        MAXCS0L
  X:F002H         PUBLIC        PW1YH
  D:00D0H         PUBLIC        PSW
  X:F016H         PUBLIC        PW2YH
  D:00AEH         PUBLIC        CRCDATH
  X:F030H         PUBLIC        PW3YH
  D:00C0H         PUBLIC        IRCON
  -------         PROC          MAIN
  -------         DO            
  D:0008H         SYMBOL        dbCRC16_OneByte_Result
  D:0006H         SYMBOL        dbCRC16_AppResult
  D:000AH         SYMBOL        dbCRC16_RANGE_ADDR
  D:0004H         SYMBOL        i
  D:000CH         SYMBOL        Addrptr
  D:000EH         SYMBOL        AddrprtCRCOption
  -------         ENDDO         
  C:0003H         LINE#         40
  C:0003H         LINE#         41
  C:0003H         LINE#         44
  C:0009H         LINE#         50
  C:000CH         LINE#         53
  C:0011H         LINE#         54
  C:0017H         LINE#         56
  C:0017H         LINE#         57
  C:0017H         LINE#         61
  C:001AH         LINE#         62
  C:001DH         LINE#         65
  C:0029H         LINE#         66
  C:0029H         LINE#         67
  C:0037H         LINE#         68
  C:003DH         LINE#         69
  C:0047H         LINE#         70
  C:004EH         LINE#         72
  C:0062H         LINE#         76
  C:006CH         LINE#         77
  C:006CH         LINE#         78
  C:0071H         LINE#         79
  C:0073H         LINE#         81
  C:0073H         LINE#         82
  C:0078H         LINE#         83
  C:0078H         LINE#         84
  -------         ENDPROC       MAIN
  -------         PROC          GPIO_INITIALIZATION
  C:007AH         LINE#         93
  C:007AH         LINE#         94
  C:007AH         LINE#         96
  C:0080H         LINE#         97
  C:0086H         LINE#         98
  C:008CH         LINE#         99
  C:0092H         LINE#         100
  -------         ENDPROC       GPIO_INITIALIZATION
BL51 BANKED LINKER/LOCATER V6.22                                                      04/27/2022  11:38:43  PAGE 5


  -------         ENDMOD        MAIN

  -------         MODULE        OPTIONS_SN8F5835
  C:7FF0H         PUBLIC        CRC_CHECK_DATA
  N:00EAH         SYMBOL        BIT16_BYPASS1P_H
  N:0001H         SYMBOL        BIT16_BYPASS1P_L
  N:0008H         SYMBOL        CK_FINE_TUNING_SET
  N:0018H         SYMBOL        CLOCKSRC_SET
  N:00C0H         SYMBOL        EXTERNAL_CLOCKRATE_SET
  N:00A0H         SYMBOL        IHRC32M_CLOCKRATE_SET
  N:0004H         SYMBOL        ISP_EN_SET
  N:0001H         SYMBOL        NOISEFILT_SET
  N:0030H         SYMBOL        RESETPIN_SET
  N:8000H         SYMBOL        ROM_SIZE
  N:0003H         SYMBOL        SECURITY_SET
  N:00C0H         SYMBOL        WATCHCLK_SET
  N:00A0H         SYMBOL        WATCHDOG_SET
  N:00C0H         SYMBOL        XTAL12M_CLOCKRATE_SET
  N:00E0H         SYMBOL        XTAL4M_CLOCKRATE_SET
  -------         ENDMOD        OPTIONS_SN8F5835

Program Size: data=17.0 xdata=50 code=171
LINK/LOCATE RUN COMPLETE.  0 WARNING(S),  0 ERROR(S)
